
D:\STM32\Program\1.11_Odchudzanie\um0427\FWLib\project\RIDE\STM3210E-EVAL\stm32f10x_fsmc.o:     file format elf32-littlearm
D:\STM32\Program\1.11_Odchudzanie\um0427\FWLib\project\RIDE\STM3210E-EVAL\stm32f10x_fsmc.o

Disassembly of section .text.FSMC_NORSRAMDeInit:

00000000 <FSMC_NORSRAMDeInit>:
FSMC_NORSRAMDeInit():
D:\STM32\Program\1.11_Odchudzanie\um0427\FWLib\library\src/stm32f10x_fsmc.c:54
   0:	b500      	push	{lr}
D:\STM32\Program\1.11_Odchudzanie\um0427\FWLib\library\src/stm32f10x_fsmc.c:59
   2:	4686      	mov	lr, r0
   4:	b928      	cbnz	r0, 12 <FSMC_NORSRAMDeInit+0x12>
D:\STM32\Program\1.11_Odchudzanie\um0427\FWLib\library\src/stm32f10x_fsmc.c:61
   6:	f243 02db 	movw	r2, #12507	; 0x30db
   a:	f04f 4320 	mov.w	r3, #2684354560	; 0xa0000000
   e:	601a      	str	r2, [r3, #0]
  10:	e005      	b.n	1e <FSMC_NORSRAMDeInit+0x1e>
D:\STM32\Program\1.11_Odchudzanie\um0427\FWLib\library\src/stm32f10x_fsmc.c:66
  12:	f243 02d2 	movw	r2, #12498	; 0x30d2
  16:	f04f 4320 	mov.w	r3, #2684354560	; 0xa0000000
  1a:	f843 2020 	str.w	r2, [r3, r0, lsl #2]
D:\STM32\Program\1.11_Odchudzanie\um0427\FWLib\library\src/stm32f10x_fsmc.c:69
  1e:	f06f 4270 	mvn.w	r2, #4026531840	; 0xf0000000
  22:	f04f 4320 	mov.w	r3, #2684354560	; 0xa0000000
  26:	f10e 0101 	add.w	r1, lr, #1	; 0x1
  2a:	f843 2021 	str.w	r2, [r3, r1, lsl #2]
D:\STM32\Program\1.11_Odchudzanie\um0427\FWLib\library\src/stm32f10x_fsmc.c:70
  2e:	f503 7382 	add.w	r3, r3, #260	; 0x104
  32:	f843 202e 	str.w	r2, [r3, lr, lsl #2]
D:\STM32\Program\1.11_Odchudzanie\um0427\FWLib\library\src/stm32f10x_fsmc.c:71
  36:	bd00      	pop	{pc}
Disassembly of section .text.FSMC_NANDDeInit:

00000000 <FSMC_NANDDeInit>:
FSMC_NANDDeInit():
D:\STM32\Program\1.11_Odchudzanie\um0427\FWLib\library\src/stm32f10x_fsmc.c:89
   0:	2810      	cmp	r0, #16
D:\STM32\Program\1.11_Odchudzanie\um0427\FWLib\library\src/stm32f10x_fsmc.c:92
   2:	bf0c      	ite	eq
   4:	4a05      	ldreq	r2, [pc, #20]	(1c <FSMC_NANDDeInit+0x1c>)
D:\STM32\Program\1.11_Odchudzanie\um0427\FWLib\library\src/stm32f10x_fsmc.c:101
   6:	4a06      	ldrne	r2, [pc, #24]	(20 <FSMC_NANDDeInit+0x20>)
   8:	2318      	movs	r3, #24
   a:	6013      	str	r3, [r2, #0]
D:\STM32\Program\1.11_Odchudzanie\um0427\FWLib\library\src/stm32f10x_fsmc.c:102
   c:	3328      	adds	r3, #40
   e:	6053      	str	r3, [r2, #4]
D:\STM32\Program\1.11_Odchudzanie\um0427\FWLib\library\src/stm32f10x_fsmc.c:103
  10:	f04f 33fc 	mov.w	r3, #4244438268	; 0xfcfcfcfc
  14:	6093      	str	r3, [r2, #8]
D:\STM32\Program\1.11_Odchudzanie\um0427\FWLib\library\src/stm32f10x_fsmc.c:104
  16:	60d3      	str	r3, [r2, #12]
D:\STM32\Program\1.11_Odchudzanie\um0427\FWLib\library\src/stm32f10x_fsmc.c:106
  18:	4770      	bx	lr
  1a:	46c0      	nop			(mov r8, r8)
  1c:	a0000060 	.word	0xa0000060
  20:	a0000080 	.word	0xa0000080
Disassembly of section .text.FSMC_PCCARDDeInit:

00000000 <FSMC_PCCARDDeInit>:
FSMC_PCCARDDeInit():
D:\STM32\Program\1.11_Odchudzanie\um0427\FWLib\library\src/stm32f10x_fsmc.c:119
   0:	4a05      	ldr	r2, [pc, #20]	(18 <FSMC_PCCARDDeInit+0x18>)
   2:	2318      	movs	r3, #24
   4:	6013      	str	r3, [r2, #0]
D:\STM32\Program\1.11_Odchudzanie\um0427\FWLib\library\src/stm32f10x_fsmc.c:120
   6:	2300      	movs	r3, #0
   8:	6053      	str	r3, [r2, #4]
D:\STM32\Program\1.11_Odchudzanie\um0427\FWLib\library\src/stm32f10x_fsmc.c:121
   a:	f103 33fc 	add.w	r3, r3, #4244438268	; 0xfcfcfcfc
   e:	6093      	str	r3, [r2, #8]
D:\STM32\Program\1.11_Odchudzanie\um0427\FWLib\library\src/stm32f10x_fsmc.c:122
  10:	60d3      	str	r3, [r2, #12]
D:\STM32\Program\1.11_Odchudzanie\um0427\FWLib\library\src/stm32f10x_fsmc.c:123
  12:	6113      	str	r3, [r2, #16]
D:\STM32\Program\1.11_Odchudzanie\um0427\FWLib\library\src/stm32f10x_fsmc.c:124
  14:	4770      	bx	lr
  16:	46c0      	nop			(mov r8, r8)
  18:	a00000a0 	.word	0xa00000a0
Disassembly of section .text.FSMC_NORSRAMInit:

00000000 <FSMC_NORSRAMInit>:
FSMC_NORSRAMInit():
D:\STM32\Program\1.11_Odchudzanie\um0427\FWLib\library\src/stm32f10x_fsmc.c:161
   0:	6881      	ldr	r1, [r0, #8]
   2:	6843      	ldr	r3, [r0, #4]
   4:	68c2      	ldr	r2, [r0, #12]
   6:	ea41 0303 	orr.w	r3, r1, r3
   a:	4313      	orrs	r3, r2
   c:	6902      	ldr	r2, [r0, #16]
D:\STM32\Program\1.11_Odchudzanie\um0427\FWLib\library\src/stm32f10x_fsmc.c:137
   e:	b5f0      	push	{r4, r5, r6, r7, lr}
D:\STM32\Program\1.11_Odchudzanie\um0427\FWLib\library\src/stm32f10x_fsmc.c:161
  10:	4313      	orrs	r3, r2
  12:	6942      	ldr	r2, [r0, #20]
  14:	6a87      	ldr	r7, [r0, #40]
  16:	4313      	orrs	r3, r2
  18:	6982      	ldr	r2, [r0, #24]
  1a:	6806      	ldr	r6, [r0, #0]
  1c:	4313      	orrs	r3, r2
  1e:	69c2      	ldr	r2, [r0, #28]
  20:	f04f 4520 	mov.w	r5, #2684354560	; 0xa0000000
  24:	4313      	orrs	r3, r2
  26:	6a02      	ldr	r2, [r0, #32]
D:\STM32\Program\1.11_Odchudzanie\um0427\FWLib\library\src/stm32f10x_fsmc.c:137
  28:	4604      	mov	r4, r0
D:\STM32\Program\1.11_Odchudzanie\um0427\FWLib\library\src/stm32f10x_fsmc.c:161
  2a:	4313      	orrs	r3, r2
  2c:	6a42      	ldr	r2, [r0, #36]
  2e:	4313      	orrs	r3, r2
  30:	6ac2      	ldr	r2, [r0, #44]
  32:	433b      	orrs	r3, r7
  34:	4313      	orrs	r3, r2
  36:	6b02      	ldr	r2, [r0, #48]
  38:	4313      	orrs	r3, r2
D:\STM32\Program\1.11_Odchudzanie\um0427\FWLib\library\src/stm32f10x_fsmc.c:175
  3a:	2908      	cmp	r1, #8
D:\STM32\Program\1.11_Odchudzanie\um0427\FWLib\library\src/stm32f10x_fsmc.c:161
  3c:	f845 3026 	str.w	r3, [r5, r6, lsl #2]
D:\STM32\Program\1.11_Odchudzanie\um0427\FWLib\library\src/stm32f10x_fsmc.c:175
  40:	d105      	bne.n	4e <FSMC_NORSRAMInit+0x4e>
D:\STM32\Program\1.11_Odchudzanie\um0427\FWLib\library\src/stm32f10x_fsmc.c:177
  42:	f855 3026 	ldr.w	r3, [r5, r6, lsl #2]
  46:	f043 0340 	orr.w	r3, r3, #64	; 0x40
  4a:	f845 3026 	str.w	r3, [r5, r6, lsl #2]
D:\STM32\Program\1.11_Odchudzanie\um0427\FWLib\library\src/stm32f10x_fsmc.c:181
  4e:	6b62      	ldr	r2, [r4, #52]
  50:	1c70      	adds	r0, r6, #1
  52:	6811      	ldr	r1, [r2, #0]
  54:	6993      	ldr	r3, [r2, #24]
  56:	430b      	orrs	r3, r1
  58:	6851      	ldr	r1, [r2, #4]
D:\STM32\Program\1.11_Odchudzanie\um0427\FWLib\library\src/stm32f10x_fsmc.c:193
  5a:	f5b7 4f80 	cmp.w	r7, #16384	; 0x4000
D:\STM32\Program\1.11_Odchudzanie\um0427\FWLib\library\src/stm32f10x_fsmc.c:181
  5e:	ea43 1301 	orr.w	r3, r3, r1, lsl #4
  62:	6891      	ldr	r1, [r2, #8]
  64:	ea43 2301 	orr.w	r3, r3, r1, lsl #8
  68:	68d1      	ldr	r1, [r2, #12]
  6a:	ea43 4301 	orr.w	r3, r3, r1, lsl #16
  6e:	6911      	ldr	r1, [r2, #16]
  70:	6952      	ldr	r2, [r2, #20]
  72:	ea43 5301 	orr.w	r3, r3, r1, lsl #20
  76:	ea43 6302 	orr.w	r3, r3, r2, lsl #24
  7a:	f845 3020 	str.w	r3, [r5, r0, lsl #2]
D:\STM32\Program\1.11_Odchudzanie\um0427\FWLib\library\src/stm32f10x_fsmc.c:193
  7e:	d116      	bne.n	ae <FSMC_NORSRAMInit+0xae>
D:\STM32\Program\1.11_Odchudzanie\um0427\FWLib\library\src/stm32f10x_fsmc.c:203
  80:	6ba2      	ldr	r2, [r4, #56]
  82:	6811      	ldr	r1, [r2, #0]
  84:	6993      	ldr	r3, [r2, #24]
  86:	430b      	orrs	r3, r1
  88:	6851      	ldr	r1, [r2, #4]
  8a:	ea43 1301 	orr.w	r3, r3, r1, lsl #4
  8e:	6891      	ldr	r1, [r2, #8]
  90:	ea43 2301 	orr.w	r3, r3, r1, lsl #8
  94:	68d1      	ldr	r1, [r2, #12]
  96:	ea43 4301 	orr.w	r3, r3, r1, lsl #16
  9a:	6911      	ldr	r1, [r2, #16]
  9c:	6952      	ldr	r2, [r2, #20]
  9e:	ea43 5301 	orr.w	r3, r3, r1, lsl #20
  a2:	ea43 6302 	orr.w	r3, r3, r2, lsl #24
  a6:	4a05      	ldr	r2, [pc, #20]	(bc <FSMC_NORSRAMInit+0xbc>)
  a8:	f842 3026 	str.w	r3, [r2, r6, lsl #2]
  ac:	e004      	b.n	b8 <FSMC_NORSRAMInit+0xb8>
D:\STM32\Program\1.11_Odchudzanie\um0427\FWLib\library\src/stm32f10x_fsmc.c:214
  ae:	4b03      	ldr	r3, [pc, #12]	(bc <FSMC_NORSRAMInit+0xbc>)
  b0:	f06f 4270 	mvn.w	r2, #4026531840	; 0xf0000000
  b4:	f843 2026 	str.w	r2, [r3, r6, lsl #2]
D:\STM32\Program\1.11_Odchudzanie\um0427\FWLib\library\src/stm32f10x_fsmc.c:216
  b8:	bdf0      	pop	{r4, r5, r6, r7, pc}
  ba:	46c0      	nop			(mov r8, r8)
  bc:	a0000104 	.word	0xa0000104
Disassembly of section .text.FSMC_NANDInit:

00000000 <FSMC_NANDInit>:
FSMC_NANDInit():
D:\STM32\Program\1.11_Odchudzanie\um0427\FWLib\library\src/stm32f10x_fsmc.c:253
   0:	6882      	ldr	r2, [r0, #8]
   2:	6843      	ldr	r3, [r0, #4]
D:\STM32\Program\1.11_Odchudzanie\um0427\FWLib\library\src/stm32f10x_fsmc.c:263
   4:	6a01      	ldr	r1, [r0, #32]
D:\STM32\Program\1.11_Odchudzanie\um0427\FWLib\library\src/stm32f10x_fsmc.c:253
   6:	4313      	orrs	r3, r2
   8:	68c2      	ldr	r2, [r0, #12]
   a:	f043 0308 	orr.w	r3, r3, #8	; 0x8
   e:	4313      	orrs	r3, r2
  10:	6902      	ldr	r2, [r0, #16]
D:\STM32\Program\1.11_Odchudzanie\um0427\FWLib\library\src/stm32f10x_fsmc.c:229
  12:	b530      	push	{r4, r5, lr}
D:\STM32\Program\1.11_Odchudzanie\um0427\FWLib\library\src/stm32f10x_fsmc.c:253
  14:	4313      	orrs	r3, r2
  16:	6942      	ldr	r2, [r0, #20]
  18:	4313      	orrs	r3, r2
  1a:	6982      	ldr	r2, [r0, #24]
  1c:	ea43 2342 	orr.w	r3, r3, r2, lsl #9
  20:	69c2      	ldr	r2, [r0, #28]
  22:	ea43 3542 	orr.w	r5, r3, r2, lsl #13
D:\STM32\Program\1.11_Odchudzanie\um0427\FWLib\library\src/stm32f10x_fsmc.c:263
  26:	688b      	ldr	r3, [r1, #8]
  28:	684a      	ldr	r2, [r1, #4]
  2a:	041b      	lsls	r3, r3, #16
  2c:	ea43 2302 	orr.w	r3, r3, r2, lsl #8
  30:	680a      	ldr	r2, [r1, #0]
  32:	4313      	orrs	r3, r2
  34:	68ca      	ldr	r2, [r1, #12]
D:\STM32\Program\1.11_Odchudzanie\um0427\FWLib\library\src/stm32f10x_fsmc.c:269
  36:	6a41      	ldr	r1, [r0, #36]
D:\STM32\Program\1.11_Odchudzanie\um0427\FWLib\library\src/stm32f10x_fsmc.c:263
  38:	ea43 6402 	orr.w	r4, r3, r2, lsl #24
D:\STM32\Program\1.11_Odchudzanie\um0427\FWLib\library\src/stm32f10x_fsmc.c:269
  3c:	688b      	ldr	r3, [r1, #8]
  3e:	684a      	ldr	r2, [r1, #4]
  40:	041b      	lsls	r3, r3, #16
  42:	ea43 2302 	orr.w	r3, r3, r2, lsl #8
  46:	680a      	ldr	r2, [r1, #0]
  48:	4313      	orrs	r3, r2
  4a:	68ca      	ldr	r2, [r1, #12]
  4c:	ea43 6202 	orr.w	r2, r3, r2, lsl #24
D:\STM32\Program\1.11_Odchudzanie\um0427\FWLib\library\src/stm32f10x_fsmc.c:274
  50:	6803      	ldr	r3, [r0, #0]
  52:	2b10      	cmp	r3, #16
D:\STM32\Program\1.11_Odchudzanie\um0427\FWLib\library\src/stm32f10x_fsmc.c:277
  54:	bf0c      	ite	eq
  56:	4b03      	ldreq	r3, [pc, #12]	(64 <FSMC_NANDInit+0x64>)
D:\STM32\Program\1.11_Odchudzanie\um0427\FWLib\library\src/stm32f10x_fsmc.c:284
  58:	4b03      	ldrne	r3, [pc, #12]	(68 <FSMC_NANDInit+0x68>)
  5a:	601d      	str	r5, [r3, #0]
D:\STM32\Program\1.11_Odchudzanie\um0427\FWLib\library\src/stm32f10x_fsmc.c:285
  5c:	609c      	str	r4, [r3, #8]
D:\STM32\Program\1.11_Odchudzanie\um0427\FWLib\library\src/stm32f10x_fsmc.c:286
  5e:	60da      	str	r2, [r3, #12]
D:\STM32\Program\1.11_Odchudzanie\um0427\FWLib\library\src/stm32f10x_fsmc.c:288
  60:	bd30      	pop	{r4, r5, pc}
  62:	46c0      	nop			(mov r8, r8)
  64:	a0000060 	.word	0xa0000060
  68:	a0000080 	.word	0xa0000080
Disassembly of section .text.FSMC_PCCARDInit:

00000000 <FSMC_PCCARDInit>:
FSMC_PCCARDInit():
D:\STM32\Program\1.11_Odchudzanie\um0427\FWLib\library\src/stm32f10x_fsmc.c:325
   0:	6802      	ldr	r2, [r0, #0]
   2:	6843      	ldr	r3, [r0, #4]
D:\STM32\Program\1.11_Odchudzanie\um0427\FWLib\library\src/stm32f10x_fsmc.c:301
   4:	b510      	push	{r4, lr}
D:\STM32\Program\1.11_Odchudzanie\um0427\FWLib\library\src/stm32f10x_fsmc.c:325
   6:	4313      	orrs	r3, r2
   8:	6882      	ldr	r2, [r0, #8]
   a:	4c16      	ldr	r4, [pc, #88]	(64 <FSMC_PCCARDInit+0x64>)
   c:	ea43 2342 	orr.w	r3, r3, r2, lsl #9
  10:	68c2      	ldr	r2, [r0, #12]
D:\STM32\Program\1.11_Odchudzanie\um0427\FWLib\library\src/stm32f10x_fsmc.c:331
  12:	6901      	ldr	r1, [r0, #16]
D:\STM32\Program\1.11_Odchudzanie\um0427\FWLib\library\src/stm32f10x_fsmc.c:325
  14:	ea43 3342 	orr.w	r3, r3, r2, lsl #13
  18:	6023      	str	r3, [r4, #0]
D:\STM32\Program\1.11_Odchudzanie\um0427\FWLib\library\src/stm32f10x_fsmc.c:331
  1a:	688b      	ldr	r3, [r1, #8]
  1c:	684a      	ldr	r2, [r1, #4]
  1e:	041b      	lsls	r3, r3, #16
  20:	ea43 2302 	orr.w	r3, r3, r2, lsl #8
  24:	680a      	ldr	r2, [r1, #0]
  26:	4313      	orrs	r3, r2
  28:	68ca      	ldr	r2, [r1, #12]
D:\STM32\Program\1.11_Odchudzanie\um0427\FWLib\library\src/stm32f10x_fsmc.c:337
  2a:	6941      	ldr	r1, [r0, #20]
D:\STM32\Program\1.11_Odchudzanie\um0427\FWLib\library\src/stm32f10x_fsmc.c:331
  2c:	ea43 6302 	orr.w	r3, r3, r2, lsl #24
  30:	60a3      	str	r3, [r4, #8]
D:\STM32\Program\1.11_Odchudzanie\um0427\FWLib\library\src/stm32f10x_fsmc.c:337
  32:	688b      	ldr	r3, [r1, #8]
  34:	684a      	ldr	r2, [r1, #4]
  36:	041b      	lsls	r3, r3, #16
  38:	ea43 2302 	orr.w	r3, r3, r2, lsl #8
  3c:	680a      	ldr	r2, [r1, #0]
  3e:	4313      	orrs	r3, r2
  40:	68ca      	ldr	r2, [r1, #12]
D:\STM32\Program\1.11_Odchudzanie\um0427\FWLib\library\src/stm32f10x_fsmc.c:343
  42:	6981      	ldr	r1, [r0, #24]
D:\STM32\Program\1.11_Odchudzanie\um0427\FWLib\library\src/stm32f10x_fsmc.c:337
  44:	ea43 6302 	orr.w	r3, r3, r2, lsl #24
  48:	60e3      	str	r3, [r4, #12]
D:\STM32\Program\1.11_Odchudzanie\um0427\FWLib\library\src/stm32f10x_fsmc.c:343
  4a:	688b      	ldr	r3, [r1, #8]
  4c:	684a      	ldr	r2, [r1, #4]
  4e:	041b      	lsls	r3, r3, #16
  50:	ea43 2302 	orr.w	r3, r3, r2, lsl #8
  54:	680a      	ldr	r2, [r1, #0]
  56:	4313      	orrs	r3, r2
  58:	68ca      	ldr	r2, [r1, #12]
  5a:	ea43 6302 	orr.w	r3, r3, r2, lsl #24
  5e:	6123      	str	r3, [r4, #16]
D:\STM32\Program\1.11_Odchudzanie\um0427\FWLib\library\src/stm32f10x_fsmc.c:347
  60:	bd10      	pop	{r4, pc}
  62:	46c0      	nop			(mov r8, r8)
  64:	a00000a0 	.word	0xa00000a0
Disassembly of section .text.FSMC_NORSRAMStructInit:

00000000 <FSMC_NORSRAMStructInit>:
FSMC_NORSRAMStructInit():
D:\STM32\Program\1.11_Odchudzanie\um0427\FWLib\library\src/stm32f10x_fsmc.c:361
   0:	2302      	movs	r3, #2
   2:	6043      	str	r3, [r0, #4]
D:\STM32\Program\1.11_Odchudzanie\um0427\FWLib\library\src/stm32f10x_fsmc.c:368
   4:	f44f 5380 	mov.w	r3, #4096	; 0x1000
   8:	6203      	str	r3, [r0, #32]
D:\STM32\Program\1.11_Odchudzanie\um0427\FWLib\library\src/stm32f10x_fsmc.c:369
   a:	18db      	adds	r3, r3, r3
   c:	6243      	str	r3, [r0, #36]
D:\STM32\Program\1.11_Odchudzanie\um0427\FWLib\library\src/stm32f10x_fsmc.c:373
   e:	6b43      	ldr	r3, [r0, #52]
D:\STM32\Program\1.11_Odchudzanie\um0427\FWLib\library\src/stm32f10x_fsmc.c:360
  10:	2100      	movs	r1, #0
D:\STM32\Program\1.11_Odchudzanie\um0427\FWLib\library\src/stm32f10x_fsmc.c:373
  12:	220f      	movs	r2, #15
D:\STM32\Program\1.11_Odchudzanie\um0427\FWLib\library\src/stm32f10x_fsmc.c:358
  14:	b510      	push	{r4, lr}
D:\STM32\Program\1.11_Odchudzanie\um0427\FWLib\library\src/stm32f10x_fsmc.c:375
  16:	24ff      	movs	r4, #255
D:\STM32\Program\1.11_Odchudzanie\um0427\FWLib\library\src/stm32f10x_fsmc.c:360
  18:	6001      	str	r1, [r0, #0]
D:\STM32\Program\1.11_Odchudzanie\um0427\FWLib\library\src/stm32f10x_fsmc.c:362
  1a:	6081      	str	r1, [r0, #8]
D:\STM32\Program\1.11_Odchudzanie\um0427\FWLib\library\src/stm32f10x_fsmc.c:363
  1c:	60c1      	str	r1, [r0, #12]
D:\STM32\Program\1.11_Odchudzanie\um0427\FWLib\library\src/stm32f10x_fsmc.c:364
  1e:	6101      	str	r1, [r0, #16]
D:\STM32\Program\1.11_Odchudzanie\um0427\FWLib\library\src/stm32f10x_fsmc.c:365
  20:	6141      	str	r1, [r0, #20]
D:\STM32\Program\1.11_Odchudzanie\um0427\FWLib\library\src/stm32f10x_fsmc.c:366
  22:	6181      	str	r1, [r0, #24]
D:\STM32\Program\1.11_Odchudzanie\um0427\FWLib\library\src/stm32f10x_fsmc.c:367
  24:	61c1      	str	r1, [r0, #28]
D:\STM32\Program\1.11_Odchudzanie\um0427\FWLib\library\src/stm32f10x_fsmc.c:370
  26:	6281      	str	r1, [r0, #40]
D:\STM32\Program\1.11_Odchudzanie\um0427\FWLib\library\src/stm32f10x_fsmc.c:371
  28:	62c1      	str	r1, [r0, #44]
D:\STM32\Program\1.11_Odchudzanie\um0427\FWLib\library\src/stm32f10x_fsmc.c:372
  2a:	6301      	str	r1, [r0, #48]
D:\STM32\Program\1.11_Odchudzanie\um0427\FWLib\library\src/stm32f10x_fsmc.c:373
  2c:	601a      	str	r2, [r3, #0]
D:\STM32\Program\1.11_Odchudzanie\um0427\FWLib\library\src/stm32f10x_fsmc.c:374
  2e:	605a      	str	r2, [r3, #4]
D:\STM32\Program\1.11_Odchudzanie\um0427\FWLib\library\src/stm32f10x_fsmc.c:375
  30:	609c      	str	r4, [r3, #8]
D:\STM32\Program\1.11_Odchudzanie\um0427\FWLib\library\src/stm32f10x_fsmc.c:376
  32:	60da      	str	r2, [r3, #12]
D:\STM32\Program\1.11_Odchudzanie\um0427\FWLib\library\src/stm32f10x_fsmc.c:377
  34:	611a      	str	r2, [r3, #16]
D:\STM32\Program\1.11_Odchudzanie\um0427\FWLib\library\src/stm32f10x_fsmc.c:378
  36:	615a      	str	r2, [r3, #20]
D:\STM32\Program\1.11_Odchudzanie\um0427\FWLib\library\src/stm32f10x_fsmc.c:379
  38:	6199      	str	r1, [r3, #24]
D:\STM32\Program\1.11_Odchudzanie\um0427\FWLib\library\src/stm32f10x_fsmc.c:380
  3a:	6b83      	ldr	r3, [r0, #56]
  3c:	601a      	str	r2, [r3, #0]
D:\STM32\Program\1.11_Odchudzanie\um0427\FWLib\library\src/stm32f10x_fsmc.c:381
  3e:	605a      	str	r2, [r3, #4]
D:\STM32\Program\1.11_Odchudzanie\um0427\FWLib\library\src/stm32f10x_fsmc.c:382
  40:	609c      	str	r4, [r3, #8]
D:\STM32\Program\1.11_Odchudzanie\um0427\FWLib\library\src/stm32f10x_fsmc.c:383
  42:	60da      	str	r2, [r3, #12]
D:\STM32\Program\1.11_Odchudzanie\um0427\FWLib\library\src/stm32f10x_fsmc.c:384
  44:	611a      	str	r2, [r3, #16]
D:\STM32\Program\1.11_Odchudzanie\um0427\FWLib\library\src/stm32f10x_fsmc.c:385
  46:	615a      	str	r2, [r3, #20]
D:\STM32\Program\1.11_Odchudzanie\um0427\FWLib\library\src/stm32f10x_fsmc.c:386
  48:	6199      	str	r1, [r3, #24]
D:\STM32\Program\1.11_Odchudzanie\um0427\FWLib\library\src/stm32f10x_fsmc.c:387
  4a:	bd10      	pop	{r4, pc}
Disassembly of section .text.FSMC_NANDStructInit:

00000000 <FSMC_NANDStructInit>:
FSMC_NANDStructInit():
D:\STM32\Program\1.11_Odchudzanie\um0427\FWLib\library\src/stm32f10x_fsmc.c:400
   0:	2310      	movs	r3, #16
   2:	6003      	str	r3, [r0, #0]
D:\STM32\Program\1.11_Odchudzanie\um0427\FWLib\library\src/stm32f10x_fsmc.c:408
   4:	6a02      	ldr	r2, [r0, #32]
D:\STM32\Program\1.11_Odchudzanie\um0427\FWLib\library\src/stm32f10x_fsmc.c:401
   6:	2300      	movs	r3, #0
   8:	6043      	str	r3, [r0, #4]
D:\STM32\Program\1.11_Odchudzanie\um0427\FWLib\library\src/stm32f10x_fsmc.c:402
   a:	6083      	str	r3, [r0, #8]
D:\STM32\Program\1.11_Odchudzanie\um0427\FWLib\library\src/stm32f10x_fsmc.c:403
   c:	60c3      	str	r3, [r0, #12]
D:\STM32\Program\1.11_Odchudzanie\um0427\FWLib\library\src/stm32f10x_fsmc.c:404
   e:	6103      	str	r3, [r0, #16]
D:\STM32\Program\1.11_Odchudzanie\um0427\FWLib\library\src/stm32f10x_fsmc.c:405
  10:	6143      	str	r3, [r0, #20]
D:\STM32\Program\1.11_Odchudzanie\um0427\FWLib\library\src/stm32f10x_fsmc.c:406
  12:	6183      	str	r3, [r0, #24]
D:\STM32\Program\1.11_Odchudzanie\um0427\FWLib\library\src/stm32f10x_fsmc.c:407
  14:	61c3      	str	r3, [r0, #28]
D:\STM32\Program\1.11_Odchudzanie\um0427\FWLib\library\src/stm32f10x_fsmc.c:408
  16:	33fc      	adds	r3, #252
  18:	6013      	str	r3, [r2, #0]
D:\STM32\Program\1.11_Odchudzanie\um0427\FWLib\library\src/stm32f10x_fsmc.c:409
  1a:	6053      	str	r3, [r2, #4]
D:\STM32\Program\1.11_Odchudzanie\um0427\FWLib\library\src/stm32f10x_fsmc.c:410
  1c:	6093      	str	r3, [r2, #8]
D:\STM32\Program\1.11_Odchudzanie\um0427\FWLib\library\src/stm32f10x_fsmc.c:411
  1e:	60d3      	str	r3, [r2, #12]
D:\STM32\Program\1.11_Odchudzanie\um0427\FWLib\library\src/stm32f10x_fsmc.c:412
  20:	6a42      	ldr	r2, [r0, #36]
  22:	6013      	str	r3, [r2, #0]
D:\STM32\Program\1.11_Odchudzanie\um0427\FWLib\library\src/stm32f10x_fsmc.c:413
  24:	6053      	str	r3, [r2, #4]
D:\STM32\Program\1.11_Odchudzanie\um0427\FWLib\library\src/stm32f10x_fsmc.c:414
  26:	6093      	str	r3, [r2, #8]
D:\STM32\Program\1.11_Odchudzanie\um0427\FWLib\library\src/stm32f10x_fsmc.c:415
  28:	60d3      	str	r3, [r2, #12]
D:\STM32\Program\1.11_Odchudzanie\um0427\FWLib\library\src/stm32f10x_fsmc.c:416
  2a:	4770      	bx	lr
Disassembly of section .text.FSMC_PCCARDStructInit:

00000000 <FSMC_PCCARDStructInit>:
FSMC_PCCARDStructInit():
D:\STM32\Program\1.11_Odchudzanie\um0427\FWLib\library\src/stm32f10x_fsmc.c:429
   0:	2300      	movs	r3, #0
D:\STM32\Program\1.11_Odchudzanie\um0427\FWLib\library\src/stm32f10x_fsmc.c:433
   2:	6902      	ldr	r2, [r0, #16]
D:\STM32\Program\1.11_Odchudzanie\um0427\FWLib\library\src/stm32f10x_fsmc.c:429
   4:	6003      	str	r3, [r0, #0]
D:\STM32\Program\1.11_Odchudzanie\um0427\FWLib\library\src/stm32f10x_fsmc.c:430
   6:	6043      	str	r3, [r0, #4]
D:\STM32\Program\1.11_Odchudzanie\um0427\FWLib\library\src/stm32f10x_fsmc.c:431
   8:	6083      	str	r3, [r0, #8]
D:\STM32\Program\1.11_Odchudzanie\um0427\FWLib\library\src/stm32f10x_fsmc.c:432
   a:	60c3      	str	r3, [r0, #12]
D:\STM32\Program\1.11_Odchudzanie\um0427\FWLib\library\src/stm32f10x_fsmc.c:433
   c:	33fc      	adds	r3, #252
   e:	6013      	str	r3, [r2, #0]
D:\STM32\Program\1.11_Odchudzanie\um0427\FWLib\library\src/stm32f10x_fsmc.c:434
  10:	6053      	str	r3, [r2, #4]
D:\STM32\Program\1.11_Odchudzanie\um0427\FWLib\library\src/stm32f10x_fsmc.c:435
  12:	6093      	str	r3, [r2, #8]
D:\STM32\Program\1.11_Odchudzanie\um0427\FWLib\library\src/stm32f10x_fsmc.c:436
  14:	60d3      	str	r3, [r2, #12]
D:\STM32\Program\1.11_Odchudzanie\um0427\FWLib\library\src/stm32f10x_fsmc.c:437
  16:	6942      	ldr	r2, [r0, #20]
  18:	6013      	str	r3, [r2, #0]
D:\STM32\Program\1.11_Odchudzanie\um0427\FWLib\library\src/stm32f10x_fsmc.c:438
  1a:	6053      	str	r3, [r2, #4]
D:\STM32\Program\1.11_Odchudzanie\um0427\FWLib\library\src/stm32f10x_fsmc.c:439
  1c:	6093      	str	r3, [r2, #8]
D:\STM32\Program\1.11_Odchudzanie\um0427\FWLib\library\src/stm32f10x_fsmc.c:440
  1e:	60d3      	str	r3, [r2, #12]
D:\STM32\Program\1.11_Odchudzanie\um0427\FWLib\library\src/stm32f10x_fsmc.c:441
  20:	6982      	ldr	r2, [r0, #24]
  22:	6013      	str	r3, [r2, #0]
D:\STM32\Program\1.11_Odchudzanie\um0427\FWLib\library\src/stm32f10x_fsmc.c:442
  24:	6053      	str	r3, [r2, #4]
D:\STM32\Program\1.11_Odchudzanie\um0427\FWLib\library\src/stm32f10x_fsmc.c:443
  26:	6093      	str	r3, [r2, #8]
D:\STM32\Program\1.11_Odchudzanie\um0427\FWLib\library\src/stm32f10x_fsmc.c:444
  28:	60d3      	str	r3, [r2, #12]
D:\STM32\Program\1.11_Odchudzanie\um0427\FWLib\library\src/stm32f10x_fsmc.c:445
  2a:	4770      	bx	lr
Disassembly of section .text.FSMC_NORSRAMCmd:

00000000 <FSMC_NORSRAMCmd>:
FSMC_NORSRAMCmd():
D:\STM32\Program\1.11_Odchudzanie\um0427\FWLib\library\src/stm32f10x_fsmc.c:466
   0:	b141      	cbz	r1, 14 <FSMC_NORSRAMCmd+0x14>
D:\STM32\Program\1.11_Odchudzanie\um0427\FWLib\library\src/stm32f10x_fsmc.c:469
   2:	f04f 4220 	mov.w	r2, #2684354560	; 0xa0000000
   6:	f852 3020 	ldr.w	r3, [r2, r0, lsl #2]
   a:	f043 0301 	orr.w	r3, r3, #1	; 0x1
   e:	f842 3020 	str.w	r3, [r2, r0, lsl #2]
  12:	e008      	b.n	26 <FSMC_NORSRAMCmd+0x26>
D:\STM32\Program\1.11_Odchudzanie\um0427\FWLib\library\src/stm32f10x_fsmc.c:474
  14:	f04f 4120 	mov.w	r1, #2684354560	; 0xa0000000
  18:	f851 2020 	ldr.w	r2, [r1, r0, lsl #2]
  1c:	4b02      	ldr	r3, [pc, #8]	(28 <FSMC_NORSRAMCmd+0x28>)
  1e:	ea02 0303 	and.w	r3, r2, r3
  22:	f841 3020 	str.w	r3, [r1, r0, lsl #2]
D:\STM32\Program\1.11_Odchudzanie\um0427\FWLib\library\src/stm32f10x_fsmc.c:476
  26:	4770      	bx	lr
  28:	000ffffe 	.word	0x000ffffe
Disassembly of section .text.FSMC_NANDCmd:

00000000 <FSMC_NANDCmd>:
FSMC_NANDCmd():
D:\STM32\Program\1.11_Odchudzanie\um0427\FWLib\library\src/stm32f10x_fsmc.c:495
   0:	b141      	cbz	r1, 14 <FSMC_NANDCmd+0x14>
D:\STM32\Program\1.11_Odchudzanie\um0427\FWLib\library\src/stm32f10x_fsmc.c:498
   2:	2810      	cmp	r0, #16
D:\STM32\Program\1.11_Odchudzanie\um0427\FWLib\library\src/stm32f10x_fsmc.c:500
   4:	bf0c      	ite	eq
   6:	4a08      	ldreq	r2, [pc, #32]	(28 <FSMC_NANDCmd+0x28>)
D:\STM32\Program\1.11_Odchudzanie\um0427\FWLib\library\src/stm32f10x_fsmc.c:504
   8:	4a08      	ldrne	r2, [pc, #32]	(2c <FSMC_NANDCmd+0x2c>)
   a:	6813      	ldr	r3, [r2, #0]
   c:	f043 0304 	orr.w	r3, r3, #4	; 0x4
  10:	6013      	str	r3, [r2, #0]
  12:	e008      	b.n	26 <FSMC_NANDCmd+0x26>
D:\STM32\Program\1.11_Odchudzanie\um0427\FWLib\library\src/stm32f10x_fsmc.c:510
  14:	2810      	cmp	r0, #16
D:\STM32\Program\1.11_Odchudzanie\um0427\FWLib\library\src/stm32f10x_fsmc.c:512
  16:	bf0c      	ite	eq
  18:	4903      	ldreq	r1, [pc, #12]	(28 <FSMC_NANDCmd+0x28>)
D:\STM32\Program\1.11_Odchudzanie\um0427\FWLib\library\src/stm32f10x_fsmc.c:516
  1a:	4904      	ldrne	r1, [pc, #16]	(2c <FSMC_NANDCmd+0x2c>)
  1c:	4b04      	ldr	r3, [pc, #16]	(30 <FSMC_NANDCmd+0x30>)
  1e:	680a      	ldr	r2, [r1, #0]
  20:	ea02 0303 	and.w	r3, r2, r3
  24:	600b      	str	r3, [r1, #0]
D:\STM32\Program\1.11_Odchudzanie\um0427\FWLib\library\src/stm32f10x_fsmc.c:519
  26:	4770      	bx	lr
  28:	a0000060 	.word	0xa0000060
  2c:	a0000080 	.word	0xa0000080
  30:	000ffffb 	.word	0x000ffffb
Disassembly of section .text.FSMC_PCCARDCmd:

00000000 <FSMC_PCCARDCmd>:
FSMC_PCCARDCmd():
D:\STM32\Program\1.11_Odchudzanie\um0427\FWLib\library\src/stm32f10x_fsmc.c:533
   0:	b128      	cbz	r0, e <FSMC_PCCARDCmd+0xe>
D:\STM32\Program\1.11_Odchudzanie\um0427\FWLib\library\src/stm32f10x_fsmc.c:536
   2:	4a06      	ldr	r2, [pc, #24]	(1c <FSMC_PCCARDCmd+0x1c>)
   4:	6813      	ldr	r3, [r2, #0]
   6:	f043 0304 	orr.w	r3, r3, #4	; 0x4
   a:	6013      	str	r3, [r2, #0]
   c:	e005      	b.n	1a <FSMC_PCCARDCmd+0x1a>
D:\STM32\Program\1.11_Odchudzanie\um0427\FWLib\library\src/stm32f10x_fsmc.c:541
   e:	4903      	ldr	r1, [pc, #12]	(1c <FSMC_PCCARDCmd+0x1c>)
  10:	4b03      	ldr	r3, [pc, #12]	(20 <FSMC_PCCARDCmd+0x20>)
  12:	680a      	ldr	r2, [r1, #0]
  14:	ea02 0303 	and.w	r3, r2, r3
  18:	600b      	str	r3, [r1, #0]
D:\STM32\Program\1.11_Odchudzanie\um0427\FWLib\library\src/stm32f10x_fsmc.c:543
  1a:	4770      	bx	lr
  1c:	a00000a0 	.word	0xa00000a0
  20:	000ffffb 	.word	0x000ffffb
Disassembly of section .text.FSMC_NANDECCCmd:

00000000 <FSMC_NANDECCCmd>:
FSMC_NANDECCCmd():
D:\STM32\Program\1.11_Odchudzanie\um0427\FWLib\library\src/stm32f10x_fsmc.c:562
   0:	b141      	cbz	r1, 14 <FSMC_NANDECCCmd+0x14>
D:\STM32\Program\1.11_Odchudzanie\um0427\FWLib\library\src/stm32f10x_fsmc.c:565
   2:	2810      	cmp	r0, #16
D:\STM32\Program\1.11_Odchudzanie\um0427\FWLib\library\src/stm32f10x_fsmc.c:567
   4:	bf0c      	ite	eq
   6:	4a08      	ldreq	r2, [pc, #32]	(28 <FSMC_NANDECCCmd+0x28>)
D:\STM32\Program\1.11_Odchudzanie\um0427\FWLib\library\src/stm32f10x_fsmc.c:571
   8:	4a08      	ldrne	r2, [pc, #32]	(2c <FSMC_NANDECCCmd+0x2c>)
   a:	6813      	ldr	r3, [r2, #0]
   c:	f043 0340 	orr.w	r3, r3, #64	; 0x40
  10:	6013      	str	r3, [r2, #0]
  12:	e008      	b.n	26 <FSMC_NANDECCCmd+0x26>
D:\STM32\Program\1.11_Odchudzanie\um0427\FWLib\library\src/stm32f10x_fsmc.c:577
  14:	2810      	cmp	r0, #16
D:\STM32\Program\1.11_Odchudzanie\um0427\FWLib\library\src/stm32f10x_fsmc.c:579
  16:	bf0c      	ite	eq
  18:	4903      	ldreq	r1, [pc, #12]	(28 <FSMC_NANDECCCmd+0x28>)
D:\STM32\Program\1.11_Odchudzanie\um0427\FWLib\library\src/stm32f10x_fsmc.c:583
  1a:	4904      	ldrne	r1, [pc, #16]	(2c <FSMC_NANDECCCmd+0x2c>)
  1c:	4b04      	ldr	r3, [pc, #16]	(30 <FSMC_NANDECCCmd+0x30>)
  1e:	680a      	ldr	r2, [r1, #0]
  20:	ea02 0303 	and.w	r3, r2, r3
  24:	600b      	str	r3, [r1, #0]
D:\STM32\Program\1.11_Odchudzanie\um0427\FWLib\library\src/stm32f10x_fsmc.c:586
  26:	4770      	bx	lr
  28:	a0000060 	.word	0xa0000060
  2c:	a0000080 	.word	0xa0000080
  30:	000fffbf 	.word	0x000fffbf
Disassembly of section .text.FSMC_GetECC:

00000000 <FSMC_GetECC>:
FSMC_GetECC():
D:\STM32\Program\1.11_Odchudzanie\um0427\FWLib\library\src/stm32f10x_fsmc.c:602
   0:	2810      	cmp	r0, #16
D:\STM32\Program\1.11_Odchudzanie\um0427\FWLib\library\src/stm32f10x_fsmc.c:605
   2:	bf0c      	ite	eq
   4:	4b01      	ldreq	r3, [pc, #4]	(c <FSMC_GetECC+0xc>)
D:\STM32\Program\1.11_Odchudzanie\um0427\FWLib\library\src/stm32f10x_fsmc.c:610
   6:	4b02      	ldrne	r3, [pc, #8]	(10 <FSMC_GetECC+0x10>)
   8:	6958      	ldr	r0, [r3, #20]
D:\STM32\Program\1.11_Odchudzanie\um0427\FWLib\library\src/stm32f10x_fsmc.c:614
   a:	4770      	bx	lr
   c:	a0000060 	.word	0xa0000060
  10:	a0000080 	.word	0xa0000080
Disassembly of section .text.FSMC_ITConfig:

00000000 <FSMC_ITConfig>:
FSMC_ITConfig():
D:\STM32\Program\1.11_Odchudzanie\um0427\FWLib\library\src/stm32f10x_fsmc.c:641
   0:	b162      	cbz	r2, 1c <FSMC_ITConfig+0x1c>
D:\STM32\Program\1.11_Odchudzanie\um0427\FWLib\library\src/stm32f10x_fsmc.c:644
   2:	2810      	cmp	r0, #16
   4:	d101      	bne.n	a <FSMC_ITConfig+0xa>
D:\STM32\Program\1.11_Odchudzanie\um0427\FWLib\library\src/stm32f10x_fsmc.c:646
   6:	4a0f      	ldr	r2, [pc, #60]	(44 <FSMC_ITConfig+0x44>)
   8:	e004      	b.n	14 <FSMC_ITConfig+0x14>
D:\STM32\Program\1.11_Odchudzanie\um0427\FWLib\library\src/stm32f10x_fsmc.c:649
   a:	f5b0 7f80 	cmp.w	r0, #256	; 0x100
D:\STM32\Program\1.11_Odchudzanie\um0427\FWLib\library\src/stm32f10x_fsmc.c:651
   e:	bf0c      	ite	eq
  10:	4a0d      	ldreq	r2, [pc, #52]	(48 <FSMC_ITConfig+0x48>)
D:\STM32\Program\1.11_Odchudzanie\um0427\FWLib\library\src/stm32f10x_fsmc.c:656
  12:	4a0e      	ldrne	r2, [pc, #56]	(4c <FSMC_ITConfig+0x4c>)
  14:	6853      	ldr	r3, [r2, #4]
  16:	ea41 0303 	orr.w	r3, r1, r3
  1a:	e010      	b.n	3e <FSMC_ITConfig+0x3e>
D:\STM32\Program\1.11_Odchudzanie\um0427\FWLib\library\src/stm32f10x_fsmc.c:662
  1c:	2810      	cmp	r0, #16
  1e:	d104      	bne.n	2a <FSMC_ITConfig+0x2a>
D:\STM32\Program\1.11_Odchudzanie\um0427\FWLib\library\src/stm32f10x_fsmc.c:665
  20:	4a08      	ldr	r2, [pc, #32]	(44 <FSMC_ITConfig+0x44>)
  22:	6853      	ldr	r3, [r2, #4]
  24:	ea23 0301 	bic.w	r3, r3, r1
  28:	e009      	b.n	3e <FSMC_ITConfig+0x3e>
D:\STM32\Program\1.11_Odchudzanie\um0427\FWLib\library\src/stm32f10x_fsmc.c:668
  2a:	f5b0 7f80 	cmp.w	r0, #256	; 0x100
D:\STM32\Program\1.11_Odchudzanie\um0427\FWLib\library\src/stm32f10x_fsmc.c:670
  2e:	bf0c      	ite	eq
  30:	4a05      	ldreq	r2, [pc, #20]	(48 <FSMC_ITConfig+0x48>)
D:\STM32\Program\1.11_Odchudzanie\um0427\FWLib\library\src/stm32f10x_fsmc.c:675
  32:	4a06      	ldrne	r2, [pc, #24]	(4c <FSMC_ITConfig+0x4c>)
  34:	ea6f 0101 	mvn.w	r1, r1
  38:	6853      	ldr	r3, [r2, #4]
  3a:	ea01 0303 	and.w	r3, r1, r3
  3e:	6053      	str	r3, [r2, #4]
D:\STM32\Program\1.11_Odchudzanie\um0427\FWLib\library\src/stm32f10x_fsmc.c:678
  40:	4770      	bx	lr
  42:	46c0      	nop			(mov r8, r8)
  44:	a0000060 	.word	0xa0000060
  48:	a0000080 	.word	0xa0000080
  4c:	a00000a0 	.word	0xa00000a0
Disassembly of section .text.FSMC_GetFlagStatus:

00000000 <FSMC_GetFlagStatus>:
FSMC_GetFlagStatus():
D:\STM32\Program\1.11_Odchudzanie\um0427\FWLib\library\src/stm32f10x_fsmc.c:706
   0:	2810      	cmp	r0, #16
   2:	d101      	bne.n	8 <FSMC_GetFlagStatus+0x8>
D:\STM32\Program\1.11_Odchudzanie\um0427\FWLib\library\src/stm32f10x_fsmc.c:708
   4:	4b06      	ldr	r3, [pc, #24]	(20 <FSMC_GetFlagStatus+0x20>)
   6:	e004      	b.n	12 <FSMC_GetFlagStatus+0x12>
D:\STM32\Program\1.11_Odchudzanie\um0427\FWLib\library\src/stm32f10x_fsmc.c:710
   8:	f5b0 7f80 	cmp.w	r0, #256	; 0x100
D:\STM32\Program\1.11_Odchudzanie\um0427\FWLib\library\src/stm32f10x_fsmc.c:712
   c:	bf0c      	ite	eq
   e:	4b05      	ldreq	r3, [pc, #20]	(24 <FSMC_GetFlagStatus+0x24>)
D:\STM32\Program\1.11_Odchudzanie\um0427\FWLib\library\src/stm32f10x_fsmc.c:717
  10:	4b05      	ldrne	r3, [pc, #20]	(28 <FSMC_GetFlagStatus+0x28>)
  12:	685b      	ldr	r3, [r3, #4]
  14:	420b      	tst	r3, r1
D:\STM32\Program\1.11_Odchudzanie\um0427\FWLib\library\src/stm32f10x_fsmc.c:731
  16:	bf0c      	ite	eq
  18:	2000      	moveq	r0, #0
  1a:	2001      	movne	r0, #1
  1c:	4770      	bx	lr
  1e:	46c0      	nop			(mov r8, r8)
  20:	a0000060 	.word	0xa0000060
  24:	a0000080 	.word	0xa0000080
  28:	a00000a0 	.word	0xa00000a0
Disassembly of section .text.FSMC_ClearFlag:

00000000 <FSMC_ClearFlag>:
FSMC_ClearFlag():
D:\STM32\Program\1.11_Odchudzanie\um0427\FWLib\library\src/stm32f10x_fsmc.c:755
   0:	2810      	cmp	r0, #16
   2:	d104      	bne.n	e <FSMC_ClearFlag+0xe>
D:\STM32\Program\1.11_Odchudzanie\um0427\FWLib\library\src/stm32f10x_fsmc.c:757
   4:	4a08      	ldr	r2, [pc, #32]	(28 <FSMC_ClearFlag+0x28>)
   6:	6853      	ldr	r3, [r2, #4]
   8:	ea23 0301 	bic.w	r3, r3, r1
   c:	e009      	b.n	22 <FSMC_ClearFlag+0x22>
D:\STM32\Program\1.11_Odchudzanie\um0427\FWLib\library\src/stm32f10x_fsmc.c:759
   e:	f5b0 7f80 	cmp.w	r0, #256	; 0x100
D:\STM32\Program\1.11_Odchudzanie\um0427\FWLib\library\src/stm32f10x_fsmc.c:761
  12:	bf0c      	ite	eq
  14:	4a05      	ldreq	r2, [pc, #20]	(2c <FSMC_ClearFlag+0x2c>)
D:\STM32\Program\1.11_Odchudzanie\um0427\FWLib\library\src/stm32f10x_fsmc.c:766
  16:	4a06      	ldrne	r2, [pc, #24]	(30 <FSMC_ClearFlag+0x30>)
  18:	ea6f 0101 	mvn.w	r1, r1
  1c:	6853      	ldr	r3, [r2, #4]
  1e:	ea01 0303 	and.w	r3, r1, r3
  22:	6053      	str	r3, [r2, #4]
D:\STM32\Program\1.11_Odchudzanie\um0427\FWLib\library\src/stm32f10x_fsmc.c:768
  24:	4770      	bx	lr
  26:	46c0      	nop			(mov r8, r8)
  28:	a0000060 	.word	0xa0000060
  2c:	a0000080 	.word	0xa0000080
  30:	a00000a0 	.word	0xa00000a0
Disassembly of section .text.FSMC_GetITStatus:

00000000 <FSMC_GetITStatus>:
FSMC_GetITStatus():
D:\STM32\Program\1.11_Odchudzanie\um0427\FWLib\library\src/stm32f10x_fsmc.c:795
   0:	2810      	cmp	r0, #16
   2:	d101      	bne.n	8 <FSMC_GetITStatus+0x8>
D:\STM32\Program\1.11_Odchudzanie\um0427\FWLib\library\src/stm32f10x_fsmc.c:797
   4:	4b08      	ldr	r3, [pc, #32]	(28 <FSMC_GetITStatus+0x28>)
   6:	e004      	b.n	12 <FSMC_GetITStatus+0x12>
D:\STM32\Program\1.11_Odchudzanie\um0427\FWLib\library\src/stm32f10x_fsmc.c:799
   8:	f5b0 7f80 	cmp.w	r0, #256	; 0x100
D:\STM32\Program\1.11_Odchudzanie\um0427\FWLib\library\src/stm32f10x_fsmc.c:801
   c:	bf0c      	ite	eq
   e:	4b07      	ldreq	r3, [pc, #28]	(2c <FSMC_GetITStatus+0x2c>)
D:\STM32\Program\1.11_Odchudzanie\um0427\FWLib\library\src/stm32f10x_fsmc.c:806
  10:	4b07      	ldrne	r3, [pc, #28]	(30 <FSMC_GetITStatus+0x30>)
  12:	685b      	ldr	r3, [r3, #4]
D:\STM32\Program\1.11_Odchudzanie\um0427\FWLib\library\src/stm32f10x_fsmc.c:813
  14:	ea13 0001 	ands.w	r0, r3, r1
  18:	d004      	beq.n	24 <FSMC_GetITStatus+0x24>
  1a:	ea13 01d1 	ands.w	r1, r3, r1, lsr #3
  1e:	bf0c      	ite	eq
  20:	2000      	moveq	r0, #0
  22:	2001      	movne	r0, #1
D:\STM32\Program\1.11_Odchudzanie\um0427\FWLib\library\src/stm32f10x_fsmc.c:822
  24:	4770      	bx	lr
  26:	46c0      	nop			(mov r8, r8)
  28:	a0000060 	.word	0xa0000060
  2c:	a0000080 	.word	0xa0000080
  30:	a00000a0 	.word	0xa00000a0
Disassembly of section .text.FSMC_ClearITPendingBit:

00000000 <FSMC_ClearITPendingBit>:
FSMC_ClearITPendingBit():
D:\STM32\Program\1.11_Odchudzanie\um0427\FWLib\library\src/stm32f10x_fsmc.c:846
   0:	2810      	cmp	r0, #16
D:\STM32\Program\1.11_Odchudzanie\um0427\FWLib\library\src/stm32f10x_fsmc.c:841
   2:	460b      	mov	r3, r1
D:\STM32\Program\1.11_Odchudzanie\um0427\FWLib\library\src/stm32f10x_fsmc.c:846
   4:	d106      	bne.n	14 <FSMC_ClearITPendingBit+0x14>
D:\STM32\Program\1.11_Odchudzanie\um0427\FWLib\library\src/stm32f10x_fsmc.c:848
   6:	4909      	ldr	r1, [pc, #36]	(2c <FSMC_ClearITPendingBit+0x2c>)
   8:	ea6f 03d3 	mvn.w	r3, r3, lsr #3
   c:	684a      	ldr	r2, [r1, #4]
   e:	4013      	ands	r3, r2
  10:	604b      	str	r3, [r1, #4]
  12:	e00a      	b.n	2a <FSMC_ClearITPendingBit+0x2a>
D:\STM32\Program\1.11_Odchudzanie\um0427\FWLib\library\src/stm32f10x_fsmc.c:850
  14:	f5b0 7f80 	cmp.w	r0, #256	; 0x100
D:\STM32\Program\1.11_Odchudzanie\um0427\FWLib\library\src/stm32f10x_fsmc.c:852
  18:	bf0c      	ite	eq
  1a:	4a05      	ldreq	r2, [pc, #20]	(30 <FSMC_ClearITPendingBit+0x30>)
D:\STM32\Program\1.11_Odchudzanie\um0427\FWLib\library\src/stm32f10x_fsmc.c:857
  1c:	4a05      	ldrne	r2, [pc, #20]	(34 <FSMC_ClearITPendingBit+0x34>)
  1e:	ea4f 01d1 	mov.w	r1, r1, lsr #3
  22:	6853      	ldr	r3, [r2, #4]
  24:	ea23 0301 	bic.w	r3, r3, r1
  28:	6053      	str	r3, [r2, #4]
D:\STM32\Program\1.11_Odchudzanie\um0427\FWLib\library\src/stm32f10x_fsmc.c:859
  2a:	4770      	bx	lr
  2c:	a0000060 	.word	0xa0000060
  30:	a0000080 	.word	0xa0000080
  34:	a00000a0 	.word	0xa00000a0
